:020000020000FC
:1000000028C019E11A95F1F708950AE0309508948F
:1000100010F4D99802C0D99A0000F3DFF2DF3695C8
:100020000A95B1F7089509E0C899FECFEADFE9DF44
:10003000E8DF8894C89908940A9511F04795F7CF9E
:100040000895C895302D303019F0DFDF3196F9CFA3
:10005000089510E820E016BD26BD11E01EBF1FE583
:100060001DBFD99AD19ADFDFEEE6F0E0EADF6865DE
:100070006C6C6F2E667464692E34342E6563686F01
:100080002E61736D3A20796F7520747970656420E4
:0C0090000000342FBADF3AE0B8DFE5CF03
:00000001FF
